Archive member included because of file (symbol)

c:/maxim/toolchain/bin/../lib/gcc/arm-none-eabi/4.7.4/../../../../arm-none-eabi/lib/armv7e-m/fpu\libc_s.a(lib_a-__atexit2.o)
                              c:/maxim/toolchain/bin/../lib/gcc/arm-none-eabi/4.7.4/../../../../arm-none-eabi/lib/armv7e-m/fpu/crt0.o (__register_exitproc)
c:/maxim/toolchain/bin/../lib/gcc/arm-none-eabi/4.7.4/../../../../arm-none-eabi/lib/armv7e-m/fpu\libc_s.a(lib_a-exit.o)
                              c:/maxim/toolchain/bin/../lib/gcc/arm-none-eabi/4.7.4/../../../../arm-none-eabi/lib/armv7e-m/fpu/crt0.o (exit)
c:/maxim/toolchain/bin/../lib/gcc/arm-none-eabi/4.7.4/../../../../arm-none-eabi/lib/armv7e-m/fpu\libc_s.a(lib_a-fini.o)
                              c:/maxim/toolchain/bin/../lib/gcc/arm-none-eabi/4.7.4/../../../../arm-none-eabi/lib/armv7e-m/fpu/crt0.o (__libc_fini_array)
c:/maxim/toolchain/bin/../lib/gcc/arm-none-eabi/4.7.4/../../../../arm-none-eabi/lib/armv7e-m/fpu\libc_s.a(lib_a-impure.o)
                              c:/maxim/toolchain/bin/../lib/gcc/arm-none-eabi/4.7.4/../../../../arm-none-eabi/lib/armv7e-m/fpu\libc_s.a(lib_a-exit.o) (_global_impure_ptr)
c:/maxim/toolchain/bin/../lib/gcc/arm-none-eabi/4.7.4/../../../../arm-none-eabi/lib/armv7e-m/fpu\libc_s.a(lib_a-init.o)
                              c:/maxim/toolchain/bin/../lib/gcc/arm-none-eabi/4.7.4/../../../../arm-none-eabi/lib/armv7e-m/fpu/crt0.o (__libc_init_array)
c:/maxim/toolchain/bin/../lib/gcc/arm-none-eabi/4.7.4/../../../../arm-none-eabi/lib/armv7e-m/fpu\libc_s.a(lib_a-memset.o)
                              c:/maxim/toolchain/bin/../lib/gcc/arm-none-eabi/4.7.4/../../../../arm-none-eabi/lib/armv7e-m/fpu/crt0.o (memset)
c:/maxim/toolchain/bin/../lib/gcc/arm-none-eabi/4.7.4/../../../../arm-none-eabi/lib/armv7e-m/fpu\libnosys.a(_exit.o)
                              c:/maxim/toolchain/bin/../lib/gcc/arm-none-eabi/4.7.4/../../../../arm-none-eabi/lib/armv7e-m/fpu\libc_s.a(lib_a-exit.o) (_exit)

Discarded input sections

 .text          0x00000000        0x0 c:/maxim/toolchain/bin/../lib/gcc/arm-none-eabi/4.7.4/armv7e-m/fpu/crti.o
 .data          0x00000000        0x0 c:/maxim/toolchain/bin/../lib/gcc/arm-none-eabi/4.7.4/armv7e-m/fpu/crti.o
 .bss           0x00000000        0x0 c:/maxim/toolchain/bin/../lib/gcc/arm-none-eabi/4.7.4/armv7e-m/fpu/crti.o
 .data          0x00000000        0x4 c:/maxim/toolchain/bin/../lib/gcc/arm-none-eabi/4.7.4/armv7e-m/fpu/crtbegin.o
 .data          0x00000000        0x0 c:/maxim/toolchain/bin/../lib/gcc/arm-none-eabi/4.7.4/../../../../arm-none-eabi/lib/armv7e-m/fpu/crt0.o
 .bss           0x00000000        0x0 c:/maxim/toolchain/bin/../lib/gcc/arm-none-eabi/4.7.4/../../../../arm-none-eabi/lib/armv7e-m/fpu/crt0.o
 .ARM.extab     0x00000000        0x0 c:/maxim/toolchain/bin/../lib/gcc/arm-none-eabi/4.7.4/../../../../arm-none-eabi/lib/armv7e-m/fpu/crt0.o
 .text          0x00000000        0x0 c:/maxim/toolchain/bin/../lib/gcc/arm-none-eabi/4.7.4/../../../../arm-none-eabi/lib/armv7e-m/fpu\libc_s.a(lib_a-__atexit2.o)
 .data          0x00000000        0x0 c:/maxim/toolchain/bin/../lib/gcc/arm-none-eabi/4.7.4/../../../../arm-none-eabi/lib/armv7e-m/fpu\libc_s.a(lib_a-__atexit2.o)
 .bss           0x00000000        0x0 c:/maxim/toolchain/bin/../lib/gcc/arm-none-eabi/4.7.4/../../../../arm-none-eabi/lib/armv7e-m/fpu\libc_s.a(lib_a-__atexit2.o)
 .text          0x00000000        0x0 c:/maxim/toolchain/bin/../lib/gcc/arm-none-eabi/4.7.4/../../../../arm-none-eabi/lib/armv7e-m/fpu\libc_s.a(lib_a-exit.o)
 .data          0x00000000        0x0 c:/maxim/toolchain/bin/../lib/gcc/arm-none-eabi/4.7.4/../../../../arm-none-eabi/lib/armv7e-m/fpu\libc_s.a(lib_a-exit.o)
 .bss           0x00000000        0x0 c:/maxim/toolchain/bin/../lib/gcc/arm-none-eabi/4.7.4/../../../../arm-none-eabi/lib/armv7e-m/fpu\libc_s.a(lib_a-exit.o)
 .text          0x00000000        0x0 c:/maxim/toolchain/bin/../lib/gcc/arm-none-eabi/4.7.4/../../../../arm-none-eabi/lib/armv7e-m/fpu\libc_s.a(lib_a-fini.o)
 .data          0x00000000        0x0 c:/maxim/toolchain/bin/../lib/gcc/arm-none-eabi/4.7.4/../../../../arm-none-eabi/lib/armv7e-m/fpu\libc_s.a(lib_a-fini.o)
 .bss           0x00000000        0x0 c:/maxim/toolchain/bin/../lib/gcc/arm-none-eabi/4.7.4/../../../../arm-none-eabi/lib/armv7e-m/fpu\libc_s.a(lib_a-fini.o)
 .text          0x00000000        0x0 c:/maxim/toolchain/bin/../lib/gcc/arm-none-eabi/4.7.4/../../../../arm-none-eabi/lib/armv7e-m/fpu\libc_s.a(lib_a-impure.o)
 .data          0x00000000        0x0 c:/maxim/toolchain/bin/../lib/gcc/arm-none-eabi/4.7.4/../../../../arm-none-eabi/lib/armv7e-m/fpu\libc_s.a(lib_a-impure.o)
 .bss           0x00000000        0x0 c:/maxim/toolchain/bin/../lib/gcc/arm-none-eabi/4.7.4/../../../../arm-none-eabi/lib/armv7e-m/fpu\libc_s.a(lib_a-impure.o)
 .data._impure_ptr
                0x00000000        0x4 c:/maxim/toolchain/bin/../lib/gcc/arm-none-eabi/4.7.4/../../../../arm-none-eabi/lib/armv7e-m/fpu\libc_s.a(lib_a-impure.o)
 .text          0x00000000        0x0 c:/maxim/toolchain/bin/../lib/gcc/arm-none-eabi/4.7.4/../../../../arm-none-eabi/lib/armv7e-m/fpu\libc_s.a(lib_a-init.o)
 .data          0x00000000        0x0 c:/maxim/toolchain/bin/../lib/gcc/arm-none-eabi/4.7.4/../../../../arm-none-eabi/lib/armv7e-m/fpu\libc_s.a(lib_a-init.o)
 .bss           0x00000000        0x0 c:/maxim/toolchain/bin/../lib/gcc/arm-none-eabi/4.7.4/../../../../arm-none-eabi/lib/armv7e-m/fpu\libc_s.a(lib_a-init.o)
 .text          0x00000000        0x0 c:/maxim/toolchain/bin/../lib/gcc/arm-none-eabi/4.7.4/../../../../arm-none-eabi/lib/armv7e-m/fpu\libc_s.a(lib_a-memset.o)
 .data          0x00000000        0x0 c:/maxim/toolchain/bin/../lib/gcc/arm-none-eabi/4.7.4/../../../../arm-none-eabi/lib/armv7e-m/fpu\libc_s.a(lib_a-memset.o)
 .bss           0x00000000        0x0 c:/maxim/toolchain/bin/../lib/gcc/arm-none-eabi/4.7.4/../../../../arm-none-eabi/lib/armv7e-m/fpu\libc_s.a(lib_a-memset.o)
 .text          0x00000000        0x0 c:/maxim/toolchain/bin/../lib/gcc/arm-none-eabi/4.7.4/../../../../arm-none-eabi/lib/armv7e-m/fpu\libnosys.a(_exit.o)
 .data          0x00000000        0x0 c:/maxim/toolchain/bin/../lib/gcc/arm-none-eabi/4.7.4/../../../../arm-none-eabi/lib/armv7e-m/fpu\libnosys.a(_exit.o)
 .bss           0x00000000        0x0 c:/maxim/toolchain/bin/../lib/gcc/arm-none-eabi/4.7.4/../../../../arm-none-eabi/lib/armv7e-m/fpu\libnosys.a(_exit.o)
 .group         0x00000000        0x8 _build/system_nrf52.o
 .group         0x00000000        0x8 _build/system_nrf52.o
 .group         0x00000000        0x8 _build/system_nrf52.o
 .group         0x00000000        0x8 _build/system_nrf52.o
 .group         0x00000000        0x8 _build/system_nrf52.o
 .group         0x00000000        0x8 _build/system_nrf52.o
 .group         0x00000000        0x8 _build/system_nrf52.o
 .group         0x00000000        0x8 _build/system_nrf52.o
 .group         0x00000000        0x8 _build/system_nrf52.o
 .group         0x00000000        0x8 _build/system_nrf52.o
 .group         0x00000000        0x8 _build/system_nrf52.o
 .group         0x00000000        0x8 _build/system_nrf52.o
 .group         0x00000000        0x8 _build/system_nrf52.o
 .group         0x00000000        0x8 _build/system_nrf52.o
 .group         0x00000000        0x8 _build/system_nrf52.o
 .group         0x00000000        0x8 _build/system_nrf52.o
 .group         0x00000000        0x8 _build/system_nrf52.o
 .text          0x00000000        0x0 _build/system_nrf52.o
 .data          0x00000000        0x0 _build/system_nrf52.o
 .bss           0x00000000        0x0 _build/system_nrf52.o
 .group         0x00000000        0x8 _build/main.o
 .group         0x00000000        0x8 _build/main.o
 .group         0x00000000        0x8 _build/main.o
 .group         0x00000000        0x8 _build/main.o
 .group         0x00000000        0x8 _build/main.o
 .group         0x00000000        0x8 _build/main.o
 .group         0x00000000        0x8 _build/main.o
 .group         0x00000000        0x8 _build/main.o
 .group         0x00000000        0x8 _build/main.o
 .group         0x00000000        0x8 _build/main.o
 .group         0x00000000        0x8 _build/main.o
 .group         0x00000000        0x8 _build/main.o
 .group         0x00000000        0x8 _build/main.o
 .group         0x00000000        0x8 _build/main.o
 .group         0x00000000        0x8 _build/main.o
 .group         0x00000000        0x8 _build/main.o
 .group         0x00000000        0x8 _build/main.o
 .group         0x00000000        0x8 _build/main.o
 .group         0x00000000        0x8 _build/main.o
 .group         0x00000000        0x8 _build/main.o
 .text          0x00000000        0x0 _build/main.o
 .data          0x00000000        0x0 _build/main.o
 .bss           0x00000000        0x0 _build/main.o
 .debug_macro   0x00000000      0x874 _build/main.o
 .debug_macro   0x00000000       0x22 _build/main.o
 .debug_macro   0x00000000       0x3a _build/main.o
 .debug_macro   0x00000000       0x10 _build/main.o
 .debug_macro   0x00000000       0x2e _build/main.o
 .debug_macro   0x00000000       0xa3 _build/main.o
 .debug_macro   0x00000000      0x20e _build/main.o
 .debug_macro   0x00000000       0x1c _build/main.o
 .debug_macro   0x00000000       0x2d _build/main.o
 .debug_macro   0x00000000       0x3b _build/main.o
 .debug_macro   0x00000000       0x50 _build/main.o
 .debug_macro   0x00000000      0xe66 _build/main.o
 .debug_macro   0x00000000      0x3a0 _build/main.o
 .debug_macro   0x00000000    0x10245 _build/main.o
 .debug_macro   0x00000000     0x12c7 _build/main.o
 .debug_macro   0x00000000       0x7c _build/main.o
 .debug_macro   0x00000000       0x1c _build/main.o
 .group         0x00000000        0x8 _build/nrf_delay.o
 .group         0x00000000        0x8 _build/nrf_delay.o
 .group         0x00000000        0x8 _build/nrf_delay.o
 .group         0x00000000        0x8 _build/nrf_delay.o
 .group         0x00000000        0x8 _build/nrf_delay.o
 .group         0x00000000        0x8 _build/nrf_delay.o
 .group         0x00000000        0x8 _build/nrf_delay.o
 .group         0x00000000        0x8 _build/nrf_delay.o
 .group         0x00000000        0x8 _build/nrf_delay.o
 .group         0x00000000        0x8 _build/nrf_delay.o
 .group         0x00000000        0x8 _build/nrf_delay.o
 .group         0x00000000        0x8 _build/nrf_delay.o
 .group         0x00000000        0x8 _build/nrf_delay.o
 .group         0x00000000        0x8 _build/nrf_delay.o
 .group         0x00000000        0x8 _build/nrf_delay.o
 .group         0x00000000        0x8 _build/nrf_delay.o
 .group         0x00000000        0x8 _build/nrf_delay.o
 .group         0x00000000        0x8 _build/nrf_delay.o
 .group         0x00000000        0x8 _build/nrf_delay.o
 .group         0x00000000        0x8 _build/nrf_delay.o
 .group         0x00000000        0x8 _build/nrf_delay.o
 .group         0x00000000        0x8 _build/nrf_delay.o
 .group         0x00000000        0x8 _build/nrf_delay.o
 .group         0x00000000        0x8 _build/nrf_delay.o
 .group         0x00000000        0x8 _build/nrf_delay.o
 .group         0x00000000        0x8 _build/nrf_delay.o
 .group         0x00000000        0x8 _build/nrf_delay.o
 .group         0x00000000        0x8 _build/nrf_delay.o
 .group         0x00000000        0x8 _build/nrf_delay.o
 .text          0x00000000        0x0 _build/nrf_delay.o
 .data          0x00000000        0x0 _build/nrf_delay.o
 .bss           0x00000000        0x0 _build/nrf_delay.o
 .debug_macro   0x00000000      0x874 _build/nrf_delay.o
 .debug_macro   0x00000000       0x3a _build/nrf_delay.o
 .debug_macro   0x00000000       0x10 _build/nrf_delay.o
 .debug_macro   0x00000000       0x2e _build/nrf_delay.o
 .debug_macro   0x00000000       0xa3 _build/nrf_delay.o
 .debug_macro   0x00000000       0x1c _build/nrf_delay.o
 .debug_macro   0x00000000       0x2d _build/nrf_delay.o
 .debug_macro   0x00000000       0x50 _build/nrf_delay.o
 .debug_macro   0x00000000      0xe66 _build/nrf_delay.o
 .debug_macro   0x00000000      0x3a0 _build/nrf_delay.o
 .debug_macro   0x00000000    0x10245 _build/nrf_delay.o
 .debug_macro   0x00000000     0x12c7 _build/nrf_delay.o
 .debug_macro   0x00000000       0x7c _build/nrf_delay.o
 .data          0x00000000        0x0 _build/gcc_startup_nrf52.o
 .bss           0x00000000        0x0 _build/gcc_startup_nrf52.o
 .text          0x00000000        0x0 c:/maxim/toolchain/bin/../lib/gcc/arm-none-eabi/4.7.4/armv7e-m/fpu/crtend.o
 .data          0x00000000        0x0 c:/maxim/toolchain/bin/../lib/gcc/arm-none-eabi/4.7.4/armv7e-m/fpu/crtend.o
 .bss           0x00000000        0x0 c:/maxim/toolchain/bin/../lib/gcc/arm-none-eabi/4.7.4/armv7e-m/fpu/crtend.o
 .text          0x00000000        0x0 c:/maxim/toolchain/bin/../lib/gcc/arm-none-eabi/4.7.4/armv7e-m/fpu/crtn.o
 .data          0x00000000        0x0 c:/maxim/toolchain/bin/../lib/gcc/arm-none-eabi/4.7.4/armv7e-m/fpu/crtn.o
 .bss           0x00000000        0x0 c:/maxim/toolchain/bin/../lib/gcc/arm-none-eabi/4.7.4/armv7e-m/fpu/crtn.o

Memory Configuration

Name             Origin             Length             Attributes
FLASH            0x00000000         0x00080000         xr
RAM              0x20000000         0x00010000         xrw
*default*        0x00000000         0xffffffff

Linker script and memory map


.text           0x00000000      0xd98
 *(.isr_vector)
 .isr_vector    0x00000000      0x400 _build/gcc_startup_nrf52.o
                0x00000000                __isr_vector
 *(.text*)
 .text          0x00000400       0x54 c:/maxim/toolchain/bin/../lib/gcc/arm-none-eabi/4.7.4/armv7e-m/fpu/crtbegin.o
 .text          0x00000454       0x70 c:/maxim/toolchain/bin/../lib/gcc/arm-none-eabi/4.7.4/../../../../arm-none-eabi/lib/armv7e-m/fpu/crt0.o
                0x00000454                _start
                0x00000454                start
                0x00000454                _mainCRTStartup
 .text.__register_exitproc
                0x000004c4       0x14 c:/maxim/toolchain/bin/../lib/gcc/arm-none-eabi/4.7.4/../../../../arm-none-eabi/lib/armv7e-m/fpu\libc_s.a(lib_a-__atexit2.o)
                0x000004c4                __register_exitproc
 .text.exit     0x000004d8       0x2c c:/maxim/toolchain/bin/../lib/gcc/arm-none-eabi/4.7.4/../../../../arm-none-eabi/lib/armv7e-m/fpu\libc_s.a(lib_a-exit.o)
                0x000004d8                exit
 .text.__libc_fini_array
                0x00000504       0x2c c:/maxim/toolchain/bin/../lib/gcc/arm-none-eabi/4.7.4/../../../../arm-none-eabi/lib/armv7e-m/fpu\libc_s.a(lib_a-fini.o)
                0x00000504                __libc_fini_array
 .text.__libc_init_array
                0x00000530       0x4c c:/maxim/toolchain/bin/../lib/gcc/arm-none-eabi/4.7.4/../../../../arm-none-eabi/lib/armv7e-m/fpu\libc_s.a(lib_a-init.o)
                0x00000530                __libc_init_array
 .text.memset   0x0000057c       0x10 c:/maxim/toolchain/bin/../lib/gcc/arm-none-eabi/4.7.4/../../../../arm-none-eabi/lib/armv7e-m/fpu\libc_s.a(lib_a-memset.o)
                0x0000057c                memset
 .text._exit    0x0000058c        0x4 c:/maxim/toolchain/bin/../lib/gcc/arm-none-eabi/4.7.4/../../../../arm-none-eabi/lib/armv7e-m/fpu\libnosys.a(_exit.o)
                0x0000058c                _exit
 .text.NVIC_SystemReset
                0x00000590       0x34 _build/system_nrf52.o
 .text.SystemCoreClockUpdate
                0x000005c4       0x1c _build/system_nrf52.o
                0x000005c4                SystemCoreClockUpdate
 .text.SystemInit
                0x000005e0      0x318 _build/system_nrf52.o
                0x000005e0                SystemInit
 .text.errata_16
                0x000008f8       0x4c _build/system_nrf52.o
 .text.errata_31
                0x00000944       0x7c _build/system_nrf52.o
 .text.errata_32
                0x000009c0       0x4c _build/system_nrf52.o
 .text.errata_36
                0x00000a0c       0x7c _build/system_nrf52.o
 .text.errata_37
                0x00000a88       0x4c _build/system_nrf52.o
 .text.errata_57
                0x00000ad4       0x4c _build/system_nrf52.o
 .text.errata_66
                0x00000b20       0x4c _build/system_nrf52.o
 .text.nrf_gpio_cfg
                0x00000b6c       0x48 _build/main.o
 .text.nrf_gpio_cfg_output
                0x00000bb4       0x30 _build/main.o
 .text.main     0x00000be4       0xac _build/main.o
                0x00000be4                main
 .text.nrf_delay_ms
                0x00000c90       0xa4 _build/nrf_delay.o
                0x00000c90                nrf_delay_ms
 .text          0x00000d34       0x3c _build/gcc_startup_nrf52.o
                0x00000d34                Reset_Handler
                0x00000d5c                NMI_Handler
                0x00000d5e                HardFault_Handler
                0x00000d60                MemoryManagement_Handler
                0x00000d62                BusFault_Handler
                0x00000d64                UsageFault_Handler
                0x00000d66                SVC_Handler
                0x00000d68                DebugMonitor_Handler
                0x00000d6a                PendSV_Handler
                0x00000d6c                SysTick_Handler
                0x00000d6e                POWER_CLOCK_IRQHandler
                0x00000d6e                RADIO_IRQHandler
                0x00000d6e                PDM_IRQHandler
                0x00000d6e                TEMP_IRQHandler
                0x00000d6e                QDEC_IRQHandler
                0x00000d6e                TIMER3_IRQHandler
                0x00000d6e                PWM1_IRQHandler
                0x00000d6e                SPIM0_SPIS0_TWIM0_TWIS0_SPI0_TWI0_IRQHandler
                0x00000d6e                GPIOTE_IRQHandler
                0x00000d6e                UARTE0_UART0_IRQHandler
                0x00000d6e                TIMER4_IRQHandler
                0x00000d6e                I2S_IRQHandler
                0x00000d6e                SWI4_EGU4_IRQHandler
                0x00000d6e                FPU_IRQHandler
                0x00000d6e                TIMER2_IRQHandler
                0x00000d6e                TIMER1_IRQHandler
                0x00000d6e                PWM2_IRQHandler
                0x00000d6e                ECB_IRQHandler
                0x00000d6e                SPIM1_SPIS1_TWIM1_TWIS1_SPI1_TWI1_IRQHandler
                0x00000d6e                Default_Handler
                0x00000d6e                SAADC_IRQHandler
                0x00000d6e                CCM_AAR_IRQHandler
                0x00000d6e                WDT_IRQHandler
                0x00000d6e                SWI2_EGU2_IRQHandler
                0x00000d6e                SWI5_EGU5_IRQHandler
                0x00000d6e                RNG_IRQHandler
                0x00000d6e                RTC2_IRQHandler
                0x00000d6e                PWM0_IRQHandler
                0x00000d6e                SWI3_EGU3_IRQHandler
                0x00000d6e                RTC1_IRQHandler
                0x00000d6e                SWI1_EGU1_IRQHandler
                0x00000d6e                SPIM2_SPIS2_SPI2_IRQHandler
                0x00000d6e                NFCT_IRQHandler
                0x00000d6e                SWI0_EGU0_IRQHandler
                0x00000d6e                MWU_IRQHandler
                0x00000d6e                RTC0_IRQHandler
                0x00000d6e                TIMER0_IRQHandler
                0x00000d6e                COMP_LPCOMP_IRQHandler
 *(.init)
 .init          0x00000d70        0x4 c:/maxim/toolchain/bin/../lib/gcc/arm-none-eabi/4.7.4/armv7e-m/fpu/crti.o
                0x00000d70                _init
 .init          0x00000d74        0x8 c:/maxim/toolchain/bin/../lib/gcc/arm-none-eabi/4.7.4/armv7e-m/fpu/crtn.o
 *(.fini)
 .fini          0x00000d7c        0x4 c:/maxim/toolchain/bin/../lib/gcc/arm-none-eabi/4.7.4/armv7e-m/fpu/crti.o
                0x00000d7c                _fini
 .fini          0x00000d80        0x8 c:/maxim/toolchain/bin/../lib/gcc/arm-none-eabi/4.7.4/armv7e-m/fpu/crtn.o
 *crtbegin.o(.ctors)
 *crtbegin?.o(.ctors)
 *(EXCLUDE_FILE(*crtend.o *crtend?.o) .ctors)
 *(SORT(.ctors.*))
 *(.ctors)
 *crtbegin.o(.dtors)
 *crtbegin?.o(.dtors)
 *(EXCLUDE_FILE(*crtend.o *crtend?.o) .dtors)
 *(SORT(.dtors.*))
 *(.dtors)
 *(.rodata*)
 .rodata.str1.1
                0x00000d88        0x2 c:/maxim/toolchain/bin/../lib/gcc/arm-none-eabi/4.7.4/../../../../arm-none-eabi/lib/armv7e-m/fpu\libc_s.a(lib_a-impure.o)
 *fill*         0x00000d8a        0x2 00
 .rodata._global_impure_ptr
                0x00000d8c        0x4 c:/maxim/toolchain/bin/../lib/gcc/arm-none-eabi/4.7.4/../../../../arm-none-eabi/lib/armv7e-m/fpu\libc_s.a(lib_a-impure.o)
                0x00000d8c                _global_impure_ptr
 .rodata.leds_list
                0x00000d90        0x4 _build/main.o
                0x00000d90                leds_list
 *(.eh_frame*)
 .eh_frame      0x00000d94        0x0 c:/maxim/toolchain/bin/../lib/gcc/arm-none-eabi/4.7.4/armv7e-m/fpu/crtbegin.o
 .eh_frame      0x00000d94        0x4 c:/maxim/toolchain/bin/../lib/gcc/arm-none-eabi/4.7.4/armv7e-m/fpu/crtend.o

.glue_7         0x00000d98        0x0
 .glue_7        0x00000000        0x0 linker stubs

.glue_7t        0x00000d98        0x0
 .glue_7t       0x00000000        0x0 linker stubs

.vfp11_veneer   0x00000d98        0x0
 .vfp11_veneer  0x00000000        0x0 linker stubs

.v4_bx          0x00000d98        0x0
 .v4_bx         0x00000000        0x0 linker stubs

.iplt           0x00000d98        0x0
 .iplt          0x00000000        0x0 c:/maxim/toolchain/bin/../lib/gcc/arm-none-eabi/4.7.4/armv7e-m/fpu/crtbegin.o

.ARM.extab
 *(.ARM.extab* .gnu.linkonce.armextab.*)
                0x00000d98                __exidx_start = .

.ARM.exidx      0x00000d98        0x8
 *(.ARM.exidx* .gnu.linkonce.armexidx.*)
 .ARM.exidx     0x00000d98        0x8 c:/maxim/toolchain/bin/../lib/gcc/arm-none-eabi/4.7.4/../../../../arm-none-eabi/lib/armv7e-m/fpu/crt0.o
                0x00000da0                __exidx_end = .
                0x00000da0                __etext = .

.rel.dyn        0x00000da0        0x0
 .rel.iplt      0x00000000        0x0 c:/maxim/toolchain/bin/../lib/gcc/arm-none-eabi/4.7.4/armv7e-m/fpu/crtbegin.o

.data           0x20000000       0x74 load address 0x00000da0
                0x20000000                __data_start__ = .
 *(vtable)
 *(.data*)
 .data.impure_data
                0x20000000       0x64 c:/maxim/toolchain/bin/../lib/gcc/arm-none-eabi/4.7.4/../../../../arm-none-eabi/lib/armv7e-m/fpu\libc_s.a(lib_a-impure.o)
 .data.SystemCoreClock
                0x20000064        0x4 _build/system_nrf52.o
                0x20000064                SystemCoreClock
                0x20000068                . = ALIGN (0x4)
                0x20000068                PROVIDE (__preinit_array_start, .)
 *(.preinit_array)
                0x20000068                PROVIDE (__preinit_array_end, .)
                0x20000068                . = ALIGN (0x4)
                0x20000068                PROVIDE (__init_array_start, .)
 *(SORT(.init_array.*))
 *(.init_array)
 .init_array    0x20000068        0x4 c:/maxim/toolchain/bin/../lib/gcc/arm-none-eabi/4.7.4/armv7e-m/fpu/crtbegin.o
                0x2000006c                PROVIDE (__init_array_end, .)
                0x2000006c                . = ALIGN (0x4)
                0x2000006c                PROVIDE (__fini_array_start, .)
 *(SORT(.fini_array.*))
 *(.fini_array)
 .fini_array    0x2000006c        0x4 c:/maxim/toolchain/bin/../lib/gcc/arm-none-eabi/4.7.4/armv7e-m/fpu/crtbegin.o
                0x20000070                PROVIDE (__fini_array_end, .)
 *(.jcr*)
 .jcr           0x20000070        0x0 c:/maxim/toolchain/bin/../lib/gcc/arm-none-eabi/4.7.4/armv7e-m/fpu/crtbegin.o
 .jcr           0x20000070        0x4 c:/maxim/toolchain/bin/../lib/gcc/arm-none-eabi/4.7.4/armv7e-m/fpu/crtend.o
                0x20000074                . = ALIGN (0x4)
                0x20000074                __data_end__ = .
LOAD c:/maxim/toolchain/bin/../lib/gcc/arm-none-eabi/4.7.4/armv7e-m/fpu/crti.o
LOAD c:/maxim/toolchain/bin/../lib/gcc/arm-none-eabi/4.7.4/armv7e-m/fpu/crtbegin.o
LOAD c:/maxim/toolchain/bin/../lib/gcc/arm-none-eabi/4.7.4/../../../../arm-none-eabi/lib/armv7e-m/fpu/crt0.o
LOAD c:/maxim/toolchain/bin/../lib/gcc/arm-none-eabi/4.7.4/../../../../arm-none-eabi/lib/armv7e-m/fpu\libc_s.a
LOAD c:/maxim/toolchain/bin/../lib/gcc/arm-none-eabi/4.7.4/../../../../arm-none-eabi/lib/armv7e-m/fpu\libnosys.a
LOAD _build/system_nrf52.o
LOAD _build/main.o
LOAD _build/nrf_delay.o
LOAD _build/gcc_startup_nrf52.o
LOAD c:/maxim/toolchain/bin/../lib/gcc/arm-none-eabi/4.7.4/../../../../arm-none-eabi/lib/armv7e-m/fpu\libm.a
START GROUP
LOAD c:/maxim/toolchain/bin/../lib/gcc/arm-none-eabi/4.7.4/armv7e-m/fpu\libgcc.a
LOAD c:/maxim/toolchain/bin/../lib/gcc/arm-none-eabi/4.7.4/../../../../arm-none-eabi/lib/armv7e-m/fpu\libc_s.a
END GROUP
LOAD c:/maxim/toolchain/bin/../lib/gcc/arm-none-eabi/4.7.4/armv7e-m/fpu/crtend.o
LOAD c:/maxim/toolchain/bin/../lib/gcc/arm-none-eabi/4.7.4/armv7e-m/fpu/crtn.o
START GROUP
LOAD c:/maxim/toolchain/bin/../lib/gcc/arm-none-eabi/4.7.4/armv7e-m/fpu\libgcc.a
LOAD c:/maxim/toolchain/bin/../lib/gcc/arm-none-eabi/4.7.4/../../../../arm-none-eabi/lib/armv7e-m/fpu\libc.a
LOAD c:/maxim/toolchain/bin/../lib/gcc/arm-none-eabi/4.7.4/../../../../arm-none-eabi/lib/armv7e-m/fpu\libnosys.a
END GROUP

.igot.plt       0x20000074        0x0 load address 0x00000e14
 .igot.plt      0x00000000        0x0 c:/maxim/toolchain/bin/../lib/gcc/arm-none-eabi/4.7.4/armv7e-m/fpu/crtbegin.o

.fs_data        0x20000074        0x0
                0x20000074                PROVIDE (__start_fs_data, .)
 *(.fs_data)
                0x20000074                PROVIDE (__stop_fs_data, .)

.bss            0x20000074       0x1c load address 0x00000e14
                0x20000074                . = ALIGN (0x4)
                0x20000074                __bss_start__ = .
 *(.bss*)
 .bss           0x20000074       0x1c c:/maxim/toolchain/bin/../lib/gcc/arm-none-eabi/4.7.4/armv7e-m/fpu/crtbegin.o
 *(COMMON)
                0x20000090                . = ALIGN (0x4)
                0x20000090                __bss_end__ = .

.heap           0x20000090     0x2000
                0x20000090                __end__ = .
                0x20000090                PROVIDE (end, .)
 *(.heap*)
 .heap          0x20000090     0x2000 _build/gcc_startup_nrf52.o
                0x20000090                __HeapBase
                0x20002090                __HeapLimit = .

.stack_dummy    0x20000090     0x2000
 *(.stack*)
 .stack         0x20000090     0x2000 _build/gcc_startup_nrf52.o
                0x20010000                __StackTop = (ORIGIN (RAM) + 0x10000)
                0x2000e000                __StackLimit = (__StackTop - SIZEOF (.stack_dummy))
                0x20010000                PROVIDE (__stack, __StackTop)
                0x00000001                ASSERT ((__StackLimit >= __HeapLimit), region RAM overflowed with stack)
OUTPUT(_build/nrf52832_xxaa.out elf32-littlearm)

.ARM.attributes
                0x00000000       0x32
 .ARM.attributes
                0x00000000       0x24 c:/maxim/toolchain/bin/../lib/gcc/arm-none-eabi/4.7.4/armv7e-m/fpu/crti.o
 .ARM.attributes
                0x00000024       0x36 c:/maxim/toolchain/bin/../lib/gcc/arm-none-eabi/4.7.4/armv7e-m/fpu/crtbegin.o
 .ARM.attributes
                0x0000005a       0x22 c:/maxim/toolchain/bin/../lib/gcc/arm-none-eabi/4.7.4/../../../../arm-none-eabi/lib/armv7e-m/fpu/crt0.o
 .ARM.attributes
                0x0000007c       0x36 c:/maxim/toolchain/bin/../lib/gcc/arm-none-eabi/4.7.4/../../../../arm-none-eabi/lib/armv7e-m/fpu\libc_s.a(lib_a-__atexit2.o)
 .ARM.attributes
                0x000000b2       0x36 c:/maxim/toolchain/bin/../lib/gcc/arm-none-eabi/4.7.4/../../../../arm-none-eabi/lib/armv7e-m/fpu\libc_s.a(lib_a-exit.o)
 .ARM.attributes
                0x000000e8       0x36 c:/maxim/toolchain/bin/../lib/gcc/arm-none-eabi/4.7.4/../../../../arm-none-eabi/lib/armv7e-m/fpu\libc_s.a(lib_a-fini.o)
 .ARM.attributes
                0x0000011e       0x36 c:/maxim/toolchain/bin/../lib/gcc/arm-none-eabi/4.7.4/../../../../arm-none-eabi/lib/armv7e-m/fpu\libc_s.a(lib_a-impure.o)
 .ARM.attributes
                0x00000154       0x36 c:/maxim/toolchain/bin/../lib/gcc/arm-none-eabi/4.7.4/../../../../arm-none-eabi/lib/armv7e-m/fpu\libc_s.a(lib_a-init.o)
 .ARM.attributes
                0x0000018a       0x36 c:/maxim/toolchain/bin/../lib/gcc/arm-none-eabi/4.7.4/../../../../arm-none-eabi/lib/armv7e-m/fpu\libc_s.a(lib_a-memset.o)
 .ARM.attributes
                0x000001c0       0x36 c:/maxim/toolchain/bin/../lib/gcc/arm-none-eabi/4.7.4/../../../../arm-none-eabi/lib/armv7e-m/fpu\libnosys.a(_exit.o)
 .ARM.attributes
                0x000001f6       0x3b _build/system_nrf52.o
 .ARM.attributes
                0x00000231       0x3b _build/main.o
 .ARM.attributes
                0x0000026c       0x3b _build/nrf_delay.o
 .ARM.attributes
                0x000002a7       0x1c _build/gcc_startup_nrf52.o
 .ARM.attributes
                0x000002c3       0x36 c:/maxim/toolchain/bin/../lib/gcc/arm-none-eabi/4.7.4/armv7e-m/fpu/crtend.o
 .ARM.attributes
                0x000002f9       0x24 c:/maxim/toolchain/bin/../lib/gcc/arm-none-eabi/4.7.4/armv7e-m/fpu/crtn.o

.comment        0x00000000       0x70
 .comment       0x00000000       0x70 _build/system_nrf52.o
                                 0x71 (size before relaxing)
 .comment       0x00000000       0x71 _build/main.o
 .comment       0x00000000       0x71 _build/nrf_delay.o

.debug_frame    0x00000000      0x284
 .debug_frame   0x00000000       0x28 c:/maxim/toolchain/bin/../lib/gcc/arm-none-eabi/4.7.4/../../../../arm-none-eabi/lib/armv7e-m/fpu\libc_s.a(lib_a-__atexit2.o)
 .debug_frame   0x00000028       0x28 c:/maxim/toolchain/bin/../lib/gcc/arm-none-eabi/4.7.4/../../../../arm-none-eabi/lib/armv7e-m/fpu\libc_s.a(lib_a-exit.o)
 .debug_frame   0x00000050       0x2c c:/maxim/toolchain/bin/../lib/gcc/arm-none-eabi/4.7.4/../../../../arm-none-eabi/lib/armv7e-m/fpu\libc_s.a(lib_a-fini.o)
 .debug_frame   0x0000007c       0x2c c:/maxim/toolchain/bin/../lib/gcc/arm-none-eabi/4.7.4/../../../../arm-none-eabi/lib/armv7e-m/fpu\libc_s.a(lib_a-init.o)
 .debug_frame   0x000000a8       0x20 c:/maxim/toolchain/bin/../lib/gcc/arm-none-eabi/4.7.4/../../../../arm-none-eabi/lib/armv7e-m/fpu\libc_s.a(lib_a-memset.o)
 .debug_frame   0x000000c8       0x20 c:/maxim/toolchain/bin/../lib/gcc/arm-none-eabi/4.7.4/../../../../arm-none-eabi/lib/armv7e-m/fpu\libnosys.a(_exit.o)
 .debug_frame   0x000000e8      0x104 _build/system_nrf52.o
 .debug_frame   0x000001ec       0x6c _build/main.o
 .debug_frame   0x00000258       0x2c _build/nrf_delay.o

.debug_info     0x00000000     0x13c1
 .debug_info    0x00000000      0xec8 _build/system_nrf52.o
 .debug_info    0x00000ec8      0x3d3 _build/main.o
 .debug_info    0x0000129b      0x126 _build/nrf_delay.o

.debug_abbrev   0x00000000      0x3f7
 .debug_abbrev  0x00000000      0x1b6 _build/system_nrf52.o
 .debug_abbrev  0x000001b6      0x16f _build/main.o
 .debug_abbrev  0x00000325       0xd2 _build/nrf_delay.o

.debug_loc      0x00000000      0x298
 .debug_loc     0x00000000      0x1b8 _build/system_nrf52.o
 .debug_loc     0x000001b8       0xa8 _build/main.o
 .debug_loc     0x00000260       0x38 _build/nrf_delay.o

.debug_aranges  0x00000000       0xb8
 .debug_aranges
                0x00000000       0x68 _build/system_nrf52.o
 .debug_aranges
                0x00000068       0x30 _build/main.o
 .debug_aranges
                0x00000098       0x20 _build/nrf_delay.o

.debug_ranges   0x00000000       0x88
 .debug_ranges  0x00000000       0x58 _build/system_nrf52.o
 .debug_ranges  0x00000058       0x20 _build/main.o
 .debug_ranges  0x00000078       0x10 _build/nrf_delay.o

.debug_macro    0x00000000    0x142f1
 .debug_macro   0x00000000       0xf6 _build/system_nrf52.o
 .debug_macro   0x000000f6      0x874 _build/system_nrf52.o
 .debug_macro   0x0000096a       0x3a _build/system_nrf52.o
 .debug_macro   0x000009a4       0x10 _build/system_nrf52.o
 .debug_macro   0x000009b4       0x2e _build/system_nrf52.o
 .debug_macro   0x000009e2       0xa3 _build/system_nrf52.o
 .debug_macro   0x00000a85      0x20e _build/system_nrf52.o
 .debug_macro   0x00000c93       0x22 _build/system_nrf52.o
 .debug_macro   0x00000cb5       0x1c _build/system_nrf52.o
 .debug_macro   0x00000cd1       0x2d _build/system_nrf52.o
 .debug_macro   0x00000cfe       0x3b _build/system_nrf52.o
 .debug_macro   0x00000d39       0x50 _build/system_nrf52.o
 .debug_macro   0x00000d89      0xe66 _build/system_nrf52.o
 .debug_macro   0x00001bef      0x3a0 _build/system_nrf52.o
 .debug_macro   0x00001f8f    0x10245 _build/system_nrf52.o
 .debug_macro   0x000121d4     0x12c7 _build/system_nrf52.o
 .debug_macro   0x0001349b       0x7c _build/system_nrf52.o
 .debug_macro   0x00013517       0x1c _build/system_nrf52.o
 .debug_macro   0x00013533      0x117 _build/main.o
 .debug_macro   0x0001364a       0x10 _build/main.o
 .debug_macro   0x0001365a      0x280 _build/main.o
 .debug_macro   0x000138da       0x22 _build/main.o
 .debug_macro   0x000138fc      0x18e _build/nrf_delay.o
 .debug_macro   0x00013a8a       0x10 _build/nrf_delay.o
 .debug_macro   0x00013a9a       0x89 _build/nrf_delay.o
 .debug_macro   0x00013b23       0x10 _build/nrf_delay.o
 .debug_macro   0x00013b33       0x3a _build/nrf_delay.o
 .debug_macro   0x00013b6d       0x52 _build/nrf_delay.o
 .debug_macro   0x00013bbf       0x19 _build/nrf_delay.o
 .debug_macro   0x00013bd8      0x16d _build/nrf_delay.o
 .debug_macro   0x00013d45       0x10 _build/nrf_delay.o
 .debug_macro   0x00013d55       0xf5 _build/nrf_delay.o
 .debug_macro   0x00013e4a       0x22 _build/nrf_delay.o
 .debug_macro   0x00013e6c       0x91 _build/nrf_delay.o
 .debug_macro   0x00013efd       0x16 _build/nrf_delay.o
 .debug_macro   0x00013f13      0x16d _build/nrf_delay.o
 .debug_macro   0x00014080       0x28 _build/nrf_delay.o
 .debug_macro   0x000140a8      0x214 _build/nrf_delay.o
 .debug_macro   0x000142bc       0x35 _build/nrf_delay.o

.debug_line     0x00000000      0xdcd
 .debug_line    0x00000000      0x4e8 _build/system_nrf52.o
 .debug_line    0x000004e8      0x4b5 _build/main.o
 .debug_line    0x0000099d      0x430 _build/nrf_delay.o

.debug_str      0x00000000    0x6ec2e
 .debug_str     0x00000000    0x6ba1b _build/system_nrf52.o
                              0x6c433 (size before relaxing)
 .debug_str     0x0006ba1b      0xe4a _build/main.o
                              0x6ce0e (size before relaxing)
 .debug_str     0x0006c865     0x23c9 _build/nrf_delay.o
                              0x6e399 (size before relaxing)
